:020000006B296A
:0800080009007F399400AE20CD
:100010000F399038A000B12014077F39A100B42017
:100020007F39A20030201F149B0A08007F399400FA
:10003000AE200F398038A000B12014077F39A1000D
:10004000B4207F39A20030209B030800AE200F3976
:10005000B038A0007B30A100A20130209B01080035
:10006000FF30A3000310A20DA30D0314A20DA30DD6
:100070000310A10DA20DA30D0314A10DA20DA30D3C
:100080000310A00DA10DA20DA30D1E30950004308C
:1000900058200314A30CA20CA10CA00C031C532881
:1000A00000008515552885115528950B472808000F
:1000B0009400940B5928080019089C009C0C9C0C77
:1000C0009C0C07309C051C0818388500043058200B
:1000D000060894001C080C3E8400000895001908CE
:1000E0009C201405031D892819089C201505031D53
:1000F0007C2800309A009B2819089C209400140941
:1001000095051C080C3E84001508800001309A00FB
:100110009B2819089C201505031D992819089C2067
:1001200095041C080C3E84001508800002309A00DB
:100130009B2800309A00080007399700970A96011B
:100140000314960D9703031DA128160808008312B7
:100150008900831608148312080808000030A720BD
:1001600008000130A72008000230A7200800033053
:10017000A72008008B1383128900180888008316B3
:100180008B130812081555308900AA30890088148D
:10019000081EC82808118B17831208000030A720FA
:1001A00098000F3018060319DA28980A0F309805BE
:1001B0000030BA2008000030A72098000030180650
:1001C0000319E72898030F3098050030BA2008007B
:1001D0000130A7209800980A7F3098050130BA2096
:1001E00008000130A720980098037F30980501305F
:1001F000BA2008000130A72098000C3098077F3003
:1002000098050130BA2008000130A72098000C3072
:1002100098027F3098050130BA2008000230A720EC
:1002200098007F30180603191A29980A7F3098051C
:100230000230BA2008000230A720980000301806CB
:100240000319272998037F3098050230BA20080047
:1002500098000330BA20080000301906031D322927
:10026000DB206A2901301906031D3829CE206A29AE
:1002700002301906031D3E2904216A29033019069C
:10028000031D4429FA206A2904301906031D4A294E
:10029000F1206A2905301906031D5029E8206A2932
:1002A00006301906031D56291B216A290730190635
:1002B000031D5C290E216A2908301906031D6329D4
:1002C000003028216A2909301906031D6A290130E6
:1002D00028216A2908008B13831285018601831661
:1002E00010308500FF308600533081008312940166
:1002F000950196019701980199019A019B019C0132
:100300009F01FF308C008D008E008F0090009100C7
:1003100092009300A000A100A200A3002620990152
:1003200000301B06031D9C29B720003A03199C29A5
:100330001F1C9C2926201F105C201A08003A031954
:10034000AE291A08023A0319AB29051AA8292C214B
:1003500019080520AE2919081620AE29990A40303F
:080360001906031D9C298F29D9
:0840000005000900060007009D
:02400E00C23FAF
:08420000000029007F0000000E
:104220004D004B0043004300200076002E0031007B
:104230002E0035002E00320020004A0044005000BD
:1042400020002800630029002000320030003000E8
:0242500031003B
:00000001FF
